:0800000090C0E7C7FDCFFCCF63
:10000800FBCFFACFAEC7F8CFF7CFBDC7F5CFF4CF48
:10001800F3CFF2CFF1CFF0CFEFCFEECFEDCF00009F
:10002800000041A042A1E045A3A4A5A64BA74D48C6
:100038004FA8504354A9AA58E1ABACE2ADAE62AFA9
:10004800B0B161B2B3B4E365B6B7B8B9BABBBCBDB9
:100058006FBE7063BF79E478E5C0C1E6C2C3C4C5AA
:10006800C6C7A5BDBA79B261BF6F702E20436FB302
:10007800BC6563BFBD61C7207061B77061B26FBFF7
:10008800BA6120536F6972202620434541203230DF
:100098003133B400743D004300503D20202020251A
:1000A80000C4EE20EFEEE2EEF02E003A00CAEEF0C9
:1000B800F02E00CEF2EAEB2EF0E5EBE500C3E8F116
:1000C800F2E5F02E00D1E8E3ED2E20EEF2EAEBEEB9
:1000D800EDE5EDE8FF00CFEEE2EEF0EEF220203A9B
:1000E80000C7E2F3EA00C2FBEAEBFEF7E5ED00C267
:1000F800EAEBFEF7E5ED007A503D0064473D0070FD
:10010800473D0069473D00536F69722026204345EB
:1001180041000300020026000000F894EE27ECBB23
:10012800F1E0FBBFEBBFE5BFF8E1F1BDE1BD8DE05C
:10013800A2E0BB27ED938A95E9F780E094E0A0E67A
:10014800ED930197E9F7EAE1F1E085919591009740
:1001580061F0A591B59105901590BF01F00105904A
:100168000D920197E1F7FB01F0CFEFE5EDBFE4E079
:10017800EEBFC0E6D1E078C71A93EB81EE0FEE0F21
:10018800EE0FE064C6D810E0183050F4A981BA81A7
:10019800EE27A10FBE1FEC91EA933DD01F5FF4CF6D
:1001A800E0E8B7D818814CC12897E6E0E883E9E091
:1001B800E983EA83E6E0EB83E0E0EC83ED83EE831A
:1001C800EF83A9D8ABD8EFE1E883E983EA83EB832F
:1001D800EC83ED83EE83E0E0EF83E5E0EA939ED8DD
:1001E80028960895A0D8E07FA9D89DD8E295E07F09
:1001F800A5D870C2E3E38DD8ABD8E2E38AD8E8E2A9
:1002080088D8E8E086D8E1E084D8A2D8E6E081D8AA
:10021800ECE07FD80895909AE881EA93E3DF5AC228
:100228009098E881EA93DEDF55C21A93EA8195D85F
:10023800309731F0E130A0E0FA0711F410EC01C07A
:1002480010E8E9811E0F1A93EBDF188123960895B1
:100258001A9310E0103170F4E12F7FD8E05AFE4F66
:10026800A0E2A083E12F79D8E059FE4FA0E2A08355
:100278001F5FF0CF2EC1E881E03041F4E82D6DD842
:10028800E05AFE4FA981A083839407C0E72D65D863
:10029800E059FE4FA981A0837394B0C4EF972197CA
:1002A80080E4A0E0B0E0EAE2F0E07BDA58D8E4913C
:1002B800E03009F154D8A491A03C50F050D8E49112
:1002C8004CD8E05CF040DE01AE0FBF1FEC9102C0DD
:1002D80046D8E491EA93FE01EF5BFF4FE08146D8F0
:1002E800DE01AF5BBF4FED91FD913196FE93EE932A
:1002F8003197E491DBCFEF9624960895EB81EA934A
:10030800EB81EA9392DF34D8EC91E03039F030D8C1
:10031800ED91A883B983EA937EDFF5CF91C0C798A2
:1003280051C0E89422F822FEFECFF894F8DF84ED5D
:1003380093E00197F1F7BF988BE68A95F1F7B799A3
:1003480008C080E991E00197F1F7B79B02C0689473
:1003580001C0E89420F8789408951A93A980E89445
:1003680022F822FEFECFF89410E01830A8F4D7DF68
:1003780088E08A95F1F7A0FE05C0BF9888E08A95C5
:10038800F1F701C0BF9A8BE98A95F1F7BF98EA2D7A
:10039800F2D7AE2E1F5FE9CF789418812FC4C1DF42
:1003A800EED7EEE4EFD7EED7EA93D7DFE0E6EA93AD
:1003B800D4DF0895B6DF20FE04C0E1D7E4E4EA9371
:1003C800CCDFC79ABF9A08951A93E89422F822FEC0
:1003D800FECFF89410E01830A0F4A1DF8DE08A95E4
:1003E800F1F7BF988BE18A95F1F7E92DC4D79E2ED6
:1003F800B79B02C0E0E89E2A80EA8A95F1F71F5F62
:10040800EACF789466C0C3D9092D30E03830B8F403
:10041800E0918101E027E1701E2FE02FACD70E2F6D
:10042800E0918101A8D7E0938101103031F0A091CB
:100438008101ECE8EA27E09381013F5FE7CFACD97F
:10044800249608951A936DDF20FE43C098D7EEEBEB
:1004580099D7E0938101B8DFB92CD5DFB5DFC92C76
:10046800D2DF10E0163020F4AFDFCDDF1F5FFACF08
:10047800ABDF90928001E0918001A0918101EA17A1
:1004880011F0E89420F8C7FE0EC0BB2029F4EC2D2B
:10049800E095EF5FCE2E01C0C094EB2DE095EE5FA6
:1004A800BE2E689401C0E89421F8AC2D6FD7E0E027
:1004B800F1E0DED8DF01EB2D50D7EA0FFB1FDE2E6F
:1004C800EF2EED2DFE2DAAE0B0E0AAD896D8DE2EAC
:1004D800EF2E19910895A0918201A13330F4E09193
:1004E8008201EF5FE093820120C0E0E0E0938201A7
:1004F800689423F8A0918301A93030F4E091830136
:10050800EF5FE093830105C0E0E0E0938301689426
:1005180024F8A0918301A53011F4689425F8A091DE
:100528008301A93011F4E89425F8089531D7E093B0
:10053800940131D7E0939301EBE3E0939701089599
:10054800E8810BD7309711F4E0E3C4C0E130A0E0B4
:10055800FA0711F4E1E3BEC0E230A0E0FA0711F4B3
:10056800E2E3B8C0E330A0E0FA0711F4E3E3B2C075
:10057800E430A0E0FA0711F4E4E3ACC0E530A0E011
:10058800FA0711F4E5E3A6C0E630A0E0FA0711F493
:10059800E6E3A0C0E730A0E0FA0711F4E7E39AC069
:1005A800E830A0E0FA0711F4E8E394C0E930A0E0ED
:1005B800FA0711F4E9E38EC0E031A0E0FA0711F47C
:1005C800E0E288C087C0EAD6E857F040A8EEB3E07A
:1005D800AE1BBF0BA0938F01B09390010895AEE1BD
:1005E800B0E0E0E0B3D8A1E0B0E0DDD6AFD8A2E05B
:1005F800B0E0E0919A01AAD8A3E0B0E0E0919901B7
:10060800A5D8A4E0B0E0E0919C01A0D8A5E0B0E0B6
:10061800E0919B019BD8A6E0B0E0C8D697D8A7E0A8
:10062800B0E0B9D693D8A8E0B0E0B2D68FD8A9E0A8
:10063800B0E0BFD68BD8AAE0B0E0BED687D8ABE092
:10064800B0E0BDD683D8ACE0B0E0E091A7017ED899
:10065800ADE0B0E0E091A60179D8AEE0B0E0B2D666
:1006680075D80895B29910C0B0D6AC81BD81AE17C7
:10067800BF0720F4EC81FD81319602C0EA81FB813D
:10068800EC83FD83689427F8B3990FC0EA81FB8156
:10069800AC81BD819DD620F4EC81FD81319701C0EC
:1006A80094D6EC83FD83689427F8EC81FD81269627
:1006B8000895B09902C026FE01C00CC0689426F8BF
:1006C800E88189D6AE1718F489D6EF5F01C0E0E05B
:1006D800E093890121960895B19902C026FE01C0D0
:1006E8000FC0689426F8E0E0E09389017AD6A53037
:1006F80020F4E0918A01EF5F01C0E0E0E0938A0115
:1007080070D6A03011F433FE01C013C0B29902C0F4
:10071800999901C004C068D609DF689434F8B39980
:1007280002C0989901C005C0AB98AA9AFFDE6894E8
:1007380034F857D6A13089F4EED559D629F45BD6CA
:100748005FD661D663D666D66AD639F46BD66CD6D0
:10075800E7ECF0E06BD6E093920143D6A23081F447
:10076800DAD545D621F464D65FD650D666D657D6A4
:1007780039F41CD667D6E3E6F0E058D6E0939D013D
:1007880030D6A33039F41ED65DD6E3E6F0E04ED677
:10079800E0939E0126D6A430F1F4E2E0EA9327D64E
:1007A80039F4F6D551D6EBE3F0E040D6E093960164
:1007B80036D639F4F0D548D6E9E0F0E037D6E093FC
:1007C800950147D641F4F5D547D6E0E0F0E02CD6C0
:1007D80049DFE0938C0105D6A53041F53FD607D611
:1007E80039F4EAD52FD6E4E6F0E020D6E093A50167
:1007F80016D639F4E4D528D6E8ECF0E017D6E0931D
:10080800A80127D641F4E091A7011CD6E8ECF0E056
:100818000DD6E093A701DFD5A33041F4E091A601FE
:1008280013D6E4E6F0E002D6E093A6010895E89432
:1008380033F8999902C0989B01C002C0689433F8B4
:10084800999BAB98989BAA98B19B06C0B09B04C093
:10085800B29B02C0B39927C0E0E0E0938B01A0915E
:100868008701AF3F28F4E0918701EF5FE0938701AC
:10087800A0918701A43129F42FDF689435F8C69A2E
:10088800F0D5A0918701AB3F68F0A0918801A4360C
:1008980020F4E0918801EF5F03C01EDFE2D5E0E0BD
:1008A800E093880118C0E0E0E0938801E0938701B5
:1008B800E89426F834FE0FC0A0919801AA3020F4DD
:1008C800E0919801EF5F05C0AB98AA98E89434F8D6
:1008D800E0E0E0939801089560975BD7EA89FB8987
:1008E800C4D5AE17BF0730F0AA89BB8984D5C2D555
:1008F800E8940BC0BAD5EA89FB89BCD5C4D575D6AE
:10090800EE87FF87688B798B689437F8A0E037FC0F
:10091800A1E0E0E040FCE1E0EA1719F4B9D527D7F7
:1009280049F4E0E0E093A901E093AA01E093AB0168
:10093800E093AC01A8D5B1D545D6E093A901F093D1
:10094800AA016093AB017093AC0136D5A6D5FF27F9
:100958006627772712D72CF42FD5FF276627772706
:100968000BC02AD5FAD43DD68F01F80196D54ED6BC
:1009780009D754F4F8014AD6E093A901F093AA01E3
:100988006093AB017093AC01A091A601BB27E091E5
:10099800A901F091AA016091AB017091AC0186D5D3
:1009A800EA83FB836C837D83A091A701BB276BD56A
:1009B8007DD5EA87FB876C877D8701D5CED4FF93E9
:1009C800EF93E091A301F091A40162D51FD6A5D6BB
:1009D80003D6AF91BF916AD5EE83FF836887798785
:1009E800EA81FB816C817D81AA85BB858C859D858B
:1009F800E9D5AE81BF8188859985E9D5EAE0F0E03F
:100A080060E070E064D68F01EE85FF85E093A30176
:100A1800F093A40137FA40F81123AAF4F801E1D5BC
:100A28008F0147D5A00FB11FA136E4E0BE0710F033
:100A380045D504C0F8013DD5EA0FFB1FE0938D01B1
:100A4800F0938E0110C0F801E858FF4F32D5C0D49A
:100A580020F4A4D4E01BF10B02C0E8E7F0E0E09337
:100A68008D01F0938E019AD664960895E89436F82D
:100A780021FC21C0DDD425D508F0AD9897D46DD4DC
:100A8800ED0DFE1DA0919B01B0919C01A1D408F42D
:100A9800AD9A98D462D4E9D4EA0FFB1F12D508F0B6
:100AA80013D590D45AD4ED0DFE1DDF01A4D490D4F3
:100AB80008F00AD502C0AD9A07D5089521FC1EC0DA
:100AC800A0919201A43640F0ADD4ED0DFE1DE45680
:100AD800F040DE2EEF2E12C0A5D4A4E6B0E023D657
:100AE800EA1BFB0BEED440F09DD4A4E6B0E0AE1BAD
:100AF800BF0BDA1AEB0A02C0DD24EE240895A09198
:100B08009701A13030F0E0919701E150E09397010F
:100B180032C0EBE3E0939701A0919301A03021F458
:100B2800A0919401A23008F010C033FC0CC0999930
:100B380002C0AB98AA9A989B57D4999B02C09899DF
:100B480001C001C051D4F2DC16C0A0919401A130BB
:100B580030F0E0919401E150E09394010CC0EBE394
:100B6800E0939401A0919301A13028F0E0919301C2
:100B7800E150E09393010895E0E0A9D4E0E0AAD41D
:100B8800E0E0ABD4F5D3A436E0E0BE0748F01DD4CE
:100B9800E456F040E883F983A3D4EF5F98D4F2CF0A
:100BA800E7D31A9740F011D43A97E883F9839BD496
:100BB800EF5F90D4F5CFE88190D492D4E03011F46F
:100BC800E0E185D41BC0882491D48A92E0E6F1E064
:100BD80017D494DB77249FD37A92E0E7F1E010D41E
:100BE8008DDB0895A881A33019F483D4EA81BED39C
:100BF80085D4EA81BBD387D4EA81B8D322960895F5
:100C080027DB8824772425FE04C0B29B02C0B39951
:100C180001C002C0689401C0E89431F8E0918A01EB
:100C2800E03009F074C075D439DBE2E08E2E20FE86
:100C380006C021FC04C0E8EEF3E043D408F004C089
:100C4800EA92DA9299DF01C068D453D46CD456D4AE
:100C58006AD46BD458D467D45ED365D469D41EDB08
:100C6800E9E08E2EE1EAF0E067D418DB32FC06C03A
:100C7800E0918F01F091900161D401C04ED4A09110
:100C88008F01B0919001A83EE3E0BE0741F4ECE08B
:100C98008E2E41D355D42AD453D4E0E009C0EBE0DA
:100CA8008E2E27D440D42AD43ED43FD4E091840158
:100CB800EA9346D4E9EAF0E046D4F0DA739433FCD8
:100CC8000BC0999903C0ECE340D4D5DA989903C0D6
:100CD800EEE33BD4D0DA03C0EFE337D4CCDAECE070
:100CE8007E2EE0919301EA932BDC2FD4C4DA25FE03
:100CF80004C0E3EBF0E027D4D1DAEEE07E2EE091F9
:100D08009401AAD339DF07D3E2E0EA936BDF69D312
:100D1800A13009F044C0FDD3C1DA31FE02C07FD34F
:100D280059F469D30BD4E3E08E2EE3D3FCD3E6D396
:100D3800FAD3FBD3E8D3F7D3E7E08E2EECD2F3D384
:100D4800F7D3ACDAE5EBF0E0FED3A8DA31FE02C067
:100D5800FED3F9F4A0919201A43628F063D3E456A7
:100D6800F040ECD30DC05ED3A4E6B0E0AE1BBF0BE1
:100D7800BA93AA9301DFE9E07E2EEDE2E6D37BDAAF
:100D8800EAE07E2EBBD3C7D2E5D375DABCD3C3D293
:100D980072DAEDE07E2EBFD2BED2DFD37FDA21D366
:100DA800A23099F5EBEBF0E0C7D378DAE5ECF0E0A8
:100DB800CAD374DA3DD3C2D331FE02C030D349F46A
:100DC800EAE08E2E96D3AFD399D3ADD3AED39BD3CF
:100DD800AAD3EEE08E2E9FD2A6D3AAD35FDAE6D2AC
:100DE8003BD3CADE31FE02C0B2D349F4EBE07E2E1B
:100DF80085D391D2AFD33FDA86D38DD23CDAEEE0F9
:100E08007E2E89D288D2A9D349DAEBD2A330C1F495
:100E1800EDECF0E091D342DA31FC0CC0E5E07E2E37
:100E2800D1D21AD3A9DE6AD376D294D324DA6BD37B
:100E380072D221DAE8E07E2E6ED26DD28ED32EDA0F
:100E4800D0D2A43081F5EEEDF0E076D327DA31FE8A
:100E580002C0E5D229F0E8E08E2E9DD2EA9370D345
:100E680031FE02C074D349F093D2F6D285DEEAE0AF
:100E78008E2E3CD3E2E0EA93B5DEE9EEF0E063D3F0
:100E88000DDA31FE02C0E5D271F0E8E07E2E91D293
:100E9800E03019F4EEEEF0E002C0E7EFF0E0FA938C
:100EA800EA9339D2FBD99DD2A53009F053C0EFEFB0
:100EB800F0E042D3F3D931FE02C049D359F07CD2D5
:100EC800CBD25ADEA091A501AA3008F44AD30ED39A
:100ED800C5D288DEE8E08E2EE3E0F1E02DD3DED93E
:100EE80031FE02C09CD259F06AD2B6D245DEA0913A
:100EF800A801AA3008F435D3F9D2B0D273DEE7E0FE
:100F0800F1E021D3CBD931FE02C0A3D261F0E09148
:100F1800A701A2D231DEA091A701AA3008F421D3FB
:100F2800FAD19CD25FDEE8E07E2EEBE0F1E00BD355
:100F3800B5D931FE03C04FD2A33061F0E091A601CC
:100F48008BD21ADEA091A601AA3008F40AD3E3D105
:100F580085D248DE0895C59A85E88A95F1F7C5983F
:100F6800089501D332FC0EC0A4D2A036E4E0BE0737
:100F780018F441D2A6D208F001C0EDDF02D310F474
:100F8800689422F814C0EFD2E6E0E2BFA4DA6894CD
:100F980030F8A0919F01A43120F4E0919F01EF5F08
:100FA80004C0689432F822F8E0E0E0939F01E991E8
:100FB800EFBFF991E991B991A991999189917991A5
:100FC8006991F990199009901895AA93BA93EA93A0
:100FD800FA93EFB7EA93E0E0F0E0FDBDECBDDED1B7
:100FE800FBBDEABDE89432F8E0E0E0939F01C9D286
:100FF80010F0689422F8E991EFBFF991E991B9915D
:10100800A9911895E19781E3A0E0B0E0EAE6F0E065
:10101800C8D31A9380D16AD208D91091A001E0915F
:10102800A0019BD17096A12FB1D1AE17BF07CCF408
:10103800103140F0E091A10190D17097A12FA6D175
:10104800C7D114F4E0E208C0E12F87D17097DE0120
:101058001196AE0FBF1FEC91EA935DD10CD91F5FBB
:10106800DECF1881E2960895E0E0E2BBEBEFE1BB4A
:10107800E0EFE7BBEFE8E8BBECEFE4BBE3E0E5BBA0
:10108800E6E0E2BFE3E0E3BFE0E0EFBDE3E0EEBDB2
:10109800E0E0EDBDECBDE7BDE6BDE2BDE5BDE4BD0C
:1010A800E3BDE1E1E9BFE5B7E160E5BFE5B7E260CF
:1010B800E5BFEBB7E064EBBFE0E0EAB9E0E8E8B928
:1010C800E0E0E0BFE0ECE7B9379A329A319AE0E025
:1010D800EDB9E6BFAEE1B0E02DD3E03009F03FC096
:1010E800A1E0B0E027D3E0939201A2E0B0E04ED2B5
:1010F800A3E0B0E050D28ED1A4E0B0E047D2A5E0A2
:10110800B0E049D29AD1A6E0B0E014D3E0939D01B3
:10111800A7E0B0E00FD3E0939501A8E0B0E00AD3D0
:10112800E0939601A9E0B0E005D3E0938C01AAE032
:10113800B0E000D3E093A501ABE0B0E0FBD2E093D0
:10114800A801ACE0B0E0F6D2E093A701ADE0B0E0D2
:10115800F1D2E093A601AEE0B0E0ECD222C0E4E622
:10116800E0939201E6E8F1E055D1E0E9F1E065D1DC
:10117800E4E1E0939D01E0E0E0939501E2E0E09393
:101188009601E1E0E0938C01EAE0E093A501E2E357
:10119800E093A801E6E0E093A701E2E0E093A6016E
:1011A800EEE1E0939E015DD1C69AC0D9F9D10BDA80
:1011B8007894F5D847D9FED8FCD0E03019F0C49A15
:1011C800C7D0C49817D8F0D743D8E3E08E2EEFE005
:1011D800F1E0B2D163D8E0E0E093A001E0E5E0936C
:1011E800A101E091A101A091A001AE1760F40ADF6E
:1011F800EADCE091A001EF5FE093A001ECE2F1E00E
:10120800FFD0D4D1EECF1ED920FE07C057DC10D1B5
:1012180058D110F021FE01C0AD9ACCD8F1DCD3DC56
:10122800999B02C0989901C001C0DED030FE03C06E
:10123800E89430F8FCDA23FE1FC0E89423F8E0DCD9
:10124800C2DCC498B6D0E030B9F036FE11C0A09127
:101258009101A33058F4E0919101EF5FE09391017F
:10126800C49B02C0C49801C0C49A01C0C49802C0FB
:1012780035FCC49AE89435F824FE49C02197E894CF
:1012880024F8E5E0E883A881A13038F0DBD820FC19
:1012980004C0E881E150E883F6CF8CD820FE10C066
:1012A8000DDCE4DB32FC0AC021FE04C0E0E0F0E023
:1012B800A7D002C0EA92DA920FDB01C071D102C056
:1012C8006FD102D180D91BDCE0E0E0939101A091BD
:1012D800A201A13030F0E091A201E150E093A20117
:1012E80001C0C698A0918B01AA3030F4E0918B011F
:1012F800EF5FE0938B010AC027FE03C070D9E89422
:1013080027F8E0E0E0938901E0938A0121968ECFE7
:10131800FFCFEA9385C7E1E0EA930895FE0131968D
:10132800FA93EA9329C7919A88E28A95F1F7E2B38A
:10133800EF70E2BBE2B3AE2FE8810895EA2BE2BB7F
:1013480088E28A95F1F7919888E28A95F1F70895ED
:10135800E4E6F0E0FA93EA9329C1F0E00895FE018B
:10136800EF5BFF4F0190F081E02D0895EA9383C76A
:10137800A881B9810895F1DFF595E7950895ECEC1A
:10138800EA93EBC7EA93E9D7E0E00895B0E008955F
:10139800E09196010895E09195010895E0918D01FD
:1013A800F0918E010895E09192010895E0919D01D8
:1013B8000895E0918C010895E091A5010895E091C8
:1013C800A8010895E0919E010895E881F9810895A2
:1013D800EA17FB070895A09189010895E091890112
:1013E8000895A0918A010895AA98AB9A089561D9A1
:1013F800F5DFE0300895E0919901F0919A010895A0
:10140800FA93EA930895E1E0F0E0FACFE7EEF3E02B
:10141800F7DF28C9E0939901F0939A010895DBDF7B
:10142800A1300895C0DF99CFEBDFEDCFE9DF1AC90E
:10143800E0919B01F0919C010895E0939B01F0934A
:101448009C0108958ADFF0CF88DFDADFE0E0F0E082
:10145800D7CFC1DFA230089580DFD2CFE3E0EA938F
:101468000895EDE1E093A2010895A0919901B0914A
:101478009A010895EA1BFB0B66277727EE87FF87FB
:10148800688B798B0895EE85FF8568897989089539
:10149800AE85BF85888999890895A091A901B091E1
:1014A800AA018091AB019091AC010895B4D0E5D028
:1014B8000895A0918D01B0918E010895E0E6F4E0C1
:1014C8000895DE16EF060895689436F80895E093B7
:1014D80086010895E09385010895E09384010895B5
:1014E800E09186010895E09185010895E0E0EA938E
:1014F8000895F6DFEA9324D8EA930895F4DFEA938F
:101508001FD8EA930895E0918401EA9319D8EA93E1
:101518000895ECE9F0E074DFE9CFEDE2D8DFEDE221
:10152800D9DFEDE2DACFE0E021CFECE2EA93FBCFBE
:10153800EFE9F0E065DFDACF63DFD8CF61DF1CCBFE
:10154800FFD7EA93F0CF5CDFE6CEEA93E4CE43DF41
:10155800A030089590D6ECE2F8CF8DD6EFE9F0E010
:10156800F2CFE0E1B7CF0A921A92FA926A937A938D
:101578008A939A93AA93BA93EA93FA93EFB7EA9362
:10158800089597DFAC39E0E0BE070895D3D0FE2F69
:10159800E0E00F010895CED0E0DEE00DF11D0895E2
:1015A8008DDFE0938D01F0938E010895E991F99113
:1015B800309639F080ED97E00197F1F7A8953197CB
:1015C800C9F70895EA0FFB1F681F791F0895AE0F2A
:1015D800BF1F861F971F0895EA1BFB0B680B790B2B
:1015E8000895F195E195F0400895F095609570950E
:1015F800E195FF4F6F4F7F4F0895F695E795F69564
:10160800E795F695E795F695E79508956F2F660F98
:10161800660B762F08958B2F880F880B982F0895C7
:10162800FA9FF02DEB9FF00DEA9FE02DF10D089544
:101638007A9F702D6B9F700DF89F700DE99F700D4C
:101648006A9F602D710DFB9F600D711DE89F600DF5
:10165800711D8827FA9FF02D610D781FEB9FF00D03
:10166800611D781FEA9FE02DF10D681F781F08950E
:1016780033D0D6DF0EF4B5DF08953CD0D9DF0EF4B1
:10168800B4DF08953F934F935F93002411244427B8
:10169800552730E2AA0FBB1F881F991F001C111C79
:1016A800441F551F0E1A1F0A460B570B28F40E0E1F
:1016B8001F1E461F571F01C0A1603A9559F7FD012B
:1016C800BC01D001CA015F914F913F91089512D09A
:1016D800D9DF0EF48ADF0895E894F7FF02C081DFAE
:1016E8006894B7FF06C0A095B095119600F80394CA
:1016F80000FA0895E89477FF02C077DF689497FFAF
:101708000BC00024A095B095809590951196801DEA
:10171800901D00F8039400FA0895182E862F612D65
:10172800192E972F712D1B2EBF2FF12D1A2EAE2F8C
:10173800E12D0895E199FECFFF93FFB7F894AEBB72
:10174800BFBBE09AEDB3FFBFFF910895E19B02C0D4
:10175800A895FCCF9FB7F894AEBBBFBBE09A8DB3FA
:10176800E81719F0EDBBE29AE19A9FBF08950024AB
:101778000A160B06080609060895EA17FB07680704
:1017880079070895AE17BF078607970708953A9314
:101798002A931A930A9308953B812A811981088113
:1017A8000895AC0FBD1F05900D928A95E1F7089535
:00000001FF
